:020000040800F2
:10000000D80700209D010008A5010008392100083B
:10001000A9010008AB010008AD01000800000000C4
:10002000000000000000000000000000AF01000818
:10003000B101000800000000B3010008D92F00083A
:10004000B7010008B7010008B7010008B7010008B0
:10005000B7010008B7010008B7010008B7010008A0
:10006000B7010008B7010008B701000885140008AF
:10007000B7010008B7010008B5140008B70100086F
:10008000E5140008B7010008B7010008B70100082F
:10009000B10C0008B7010008B7010008B70100085B
:1000A000B701000845300008B7010008B701000893
:1000B000B7010008B7010008B7010008B701000840
:1000C000B7010008B7010008B7010008B701000830
:1000D000B7010008B7010008F933000849340008E7
:1000E000B7010008B7010008B7010008B701000810
:1000F000B7010008B7010008B7010008B701000800
:10010000B7010008B7010008B7010008B7010008EF
:10011000B7010008AD330008B7010008B7010008B7
:1001200015150008B7010008B7010008B70100085D
:10013000B7010008B7010008B7010008B7010008BF
:10014000B7010008B7010008B7010008B7010008AF
:10015000B7010008B7010008B7010008993400088A
:10016000B7010008B7010008B7010008B70100088F
:10017000B7010008B7010008B7010008B70100087F
:10018000B7010008B7010008DFF80CD000F01CFB35
:1001900000480047D13D0008D807002006488047A6
:1001A00006480047FEE7FEE7FEE7FEE7FEE7FEE75C
:1001B000FEE7FEE7FEE7FEE7E92F000889010008F9
:1001C0002DE9FE4F804681EA0300C00F0C460090E7
:1001D00021F0004123F00045B8EB0200A94105D20F
:1001E0004046214690461C460B46024623F00040FE
:1001F000104347D0270DC7F30A00C3F30A510290FA
:10020000401A019040286BDAC3F3130040F4801BBE
:100210000098924620B10023D2EB030A63EB0B0B4C
:1002200001985946C0F14002504600F007FA0646D0
:100230000D4650465946019A00F01FFA10EB08008F
:100240006141002487EA115284EAE7731A4340D0DF
:10025000009A62B3019A012A4FEA075215DC001B8B
:1002600061EB02014FF0004202EA0752CDE9004281
:10027000001C41F5801132462B4600F056FA03B0BF
:10028000BDE8F08F40462146F9E7001B61EB020113
:10029000001C41F5801300185B412018A2F50017DF
:1002A00047EB030140EAD570B6196D4111E06D08C6
:1002B0004FEA360645EAC0754FEA0752001B61EB6C
:1002C0000201001C41F5801149084FEA3000001975
:1002D000514132462B4603B0BDE8F04F00F016BA4C
:1002E0000098012240000023D0EB020263EBE07390
:1002F000009821464FEAE074B8EB000061EB04017E
:10030000E9E783F000435BE781F0004158E72DE91E
:10031000FE4F81EA030404F0004421F00041009400
:100320004FF0000B23F0004350EA01045ED052EA84
:1003300003045BD0C3F30A54C1F30A552C44A4F25E
:10034000F3340194A0FB0254C1F3130141F4801172
:10035000C3F3130343F4801301FB024400FB034E79
:10036000840A970A44EA815447EA8357A4FB076842
:1003700002958D0A05FB07854FEA932C04FB0C546C
:100380002705029D4FEA065847EA1637B5EB0805E0
:100390006EEB070C870E920E47EA811742EA831232
:1003A000A7FB0201B6EB0B0164EB00042B0D43EA43
:1003B0000C335E1844EB1C50DA465146E7FB020151
:1003C000C5F313044FEA0B3343EA14534FEA0432E4
:1003D000019C43EA0603A4F10C040294009CCDE9BD
:1003E00000B400F0A2F903B0BDE8F08F0020014690
:1003F000F9E72DE9F04D81EA030404F0004B21F008
:10040000004514464FF0000A23F0004150EA05026F
:1004100020D054EA01021DD0C5F30A570246C5F3A5
:100420001303C1F31300C1F30A5640F4801543F4DB
:100430008013A7EB0608101BD64608F2FD3873EBB5
:10044000050002D308F1010801E092185B41B8F100
:10045000000F03DA00200146BDE8F08D00204FF4C4
:100460008011064684460EE0171B73EB050705D383
:10047000121B63EB050306434CEA010C49084FEAE3
:10048000300092185B4150EA0107EDD152EA0300B7
:1004900012D082EA040083EA0501084305D0101B4C
:1004A000AB4106D20122002306E000224FF00043B8
:1004B00002E06FF0010253101AEB06004CEB0851FA
:1004C00010EB0A0041EB0B01BDE8F04D00F01EB946
:1004D0000EB5C10F80EAE0700844CA07002140F25F
:1004E00033438DE80E000A460B4600F01EF903B0B8
:1004F00000BD0EB540F2334102910021CDE900115B
:100500000A460B4600F011F903B000BD70B5C1F307
:100510000A5201F000450024C1F3130140F2FF33F9
:1005200041F480119A4201DA002070BD40F2334359
:100530009A42A2F2334203DC524200F08EF800E00D
:1005400090402C43F1D0404270BDC1F30A5210B527
:10055000C1F3130140F2FF3341F480119A4201DAF2
:10056000002010BD40F233439A42A2F2334203DC32
:10057000524200F072F810BD904010BD00F00042F1
:1005800030F000400AD0C10D01F56071C0F31600D3
:1005900042EA0151C208400711437047002001465A
:1005A0007047000030B5041E71F1000404DB4FF009
:1005B0000044404264EB0101141E73F1000405DBAA
:1005C0001C464FF00043524263EB04038B4208BFCA
:1005D000824230BD30B5041E71F1000404DB4FF0DF
:1005E0000044404264EB0101141E73F1000405DB7A
:1005F0001C464FF00043524263EB0403994208BF8C
:10060000904230BD01F0004330B421F0004150EA87
:10061000010206D00A0DA2F56072C1F31301002A8F
:1006200002DC30BC00207047440F44EAC104C10022
:10063000E01830BC00EBC25000F031B8202A04DBD7
:10064000203A00FA02F1002070479140C2F12003E5
:1006500020FA03F3194390407047202A04DB203A24
:1006600021FA02F00021704721FA02F3D040C2F1D2
:1006700020029140084319467047202A06DBCB1719
:10068000203A41FA02F043EAE07306E041FA02F34D
:10069000D040C2F12002914008431946704700291A
:1006A000A8BF7047401C490008BF20F001007047F8
:1006B00010B4B0FA80FC00FA0CF050EA010404BF58
:1006C00010BC704749B1CCF1200421FA04F411FAAE
:1006D0000CF118BF012121430843A3EB0C01CB1DF2
:1006E0004FEA00614FEA102042BF002010BC704763
:1006F00000EBC35010440029A4BF10BC7047401C3D
:10070000490008BF20F0010010BC704710B5141E4E
:1007100073F1000408DA401C41F1000192185B41BA
:100720001A4301D120F0010010BD2DE9F04D924691
:100730009B4611B1B1FA81F202E0B0FA80F22032A8
:100740009046FFF77BFF04460F4640EA0A0041EA65
:100750000B0153465A46084313D0114653EA010091
:1007600019D0C8F140025046FFF777FF05460E4604
:10077000504659464246FFF761FF084305D0012025
:1007800004E020463946BDE8F08D0020054346EAE6
:10079000E0762C4337430A986305E40AA0EB08008F
:1007A0000022FD0A44EA47540A3002D500200146DF
:1007B000E9E7010510196941DDE9084500196941BA
:1007C000BDE8F04DA2E70000064C074D06E0E068EA
:1007D00040F0010394E8070098471034AC42F6D388
:1007E000FFF7D6FC783F0008983F00080029816891
:1007F00002D041F0010101E021F001018160704768
:10080000084B10B5D3F8042307490A40D0E9001477
:100810002143D0E90240044321431143C3F80413A8
:1008200010BD000000200140E030FCFF10B51CA00E
:1008300086B0D0E90010CDE903104FF4C6621A4922
:10084000202000F095F8194C04222146104600F0B3
:100850008FF808222146042000F08AF8144C062064
:10086000009003AB22464FF02061201500F0B8F84D
:1008700000221146382000F0FDF80E4B2246990563
:10088000081100F035F80C4A0C4908208DE80700E3
:100890000B4B142253210B4800F034F906B010BD65
:1008A00007080E0F0C0D0000001402400008024063
:1008B0000022014010640240813200082132000809
:1008C000DD240008000C00400029816802D041F4BA
:1008D000807101E021F48071816070470029816896
:1008E00002D041F4007101E021F400718160704791
:1008F00070B50D4690B01E461446012101F0E2FD90
:100900001A480021CDE902010620CDE904014FF487
:100910008060069040000790800008904011CDE96B
:1009200009010120CDE90B104C34CDE900540D91A3
:100930000E916946304600F0F3FF0C4900220C315D
:10094000304600F093FF0121304600F085FF102172
:10095000304600F0CFFE01221021304600F0CAFFE1
:100960000121304600F0DCFE10B070BDA80300206D
:100970007CB50D461446012101F0A4FD03228DF83B
:100980000420002200948DF807206946284601F0D3
:10099000B8FA7CBD30B542680F4B0C791A400B6831
:1009A00042EA04221343436082680C4B4D791A409B
:1009B000D1E9034323438C6844EA450423431343AA
:1009C0008360C26A097D22F47002491EC9B242EAFC
:1009D0000151C16230BD0000FFFEFFFCFDF7FFC00A
:1009E0002DE9F0418AB00F461E469046044601218B
:1009F000109D01F07FFD0121204601F087FD0021BF
:100A0000204601F083FD002406944FF480300994C1
:100A1000CDE9070406A8FFF7F3FE01208DF80400D6
:100A20000007CDE9020700948DF8054004948DF885
:100A3000145069464046FFF7ADFF0D4F07E0601CBC
:100A4000C2B2315D0623384600F022F8641CAC4285
:100A5000F5DB01213846FFF741FF01214046FFF752
:100A600033FF01214046FFF7C1FE0AB0BDE8F08127
:100A70000022014008B58DF800008DF801108DF8B6
:100A8000022001208DF80300684601F0D5FC08BD66
:100A900070B5072609290AD9C568A1F10A0404EB33
:100AA0004404A640B543A3401D43C56007E0056963
:100AB00001EB4104A640B543A3401D4305611F233C
:100AC000072A09D2446B521E02EB820293409C43D8
:100AD00091400C43446370BD0D2A09D2046BD21FB0
:100AE00002EB820293409C4391400C43046370BD2F
:100AF000C46A0D3A02EB820293409C4391400C433E
:100B0000C46270BD2DE9F04188B08046DDE90E0673
:100B10000F4614460121109D98470020ADF8007043
:100B2000ADF80800ADF802008DF80A00019469469E
:100B3000404602F0FDFB0A2005906020ADF80C0055
:100B40000120ADF80E000220ADF8180003A94046C0
:100B5000B04708214046A8470121404602F003FB68
:100B60003021404602F0DCFB0121404602F0F1FA60
:100B700008B0BDE8F08100001E4800B59FED1C0ADA
:100B8000012180ED000A9FED1C0A80ED010A9FED16
:100B90001B0A80ED020A0C30B2EE0E0A80ED010A4B
:100BA0009FED170A80ED000AB0EE040A80ED030AFB
:100BB000B0EE0C0A80ED020A9FED120A80ED040AE5
:100BC000A0F53B7002F06EF802210F4802F06AF8BF
:100BD0000D480921B83002F065F806480A21B838F6
:100BE00002F060F8094801218162C16200BD000085
:100BF0009A99193F880300209A99993E00000000B5
:100C00000000964300008C4260010020000000209C
:100C100010B5044690F872000A283FD1092104F16A
:100C2000680003F0C5F894F87110884236D194F842
:100C30006800DFED1C0A00EE100AB8EE400A84EDF1
:100C40001E0AB4F8690040BA00EE100AB8EE400A75
:100C500080EE201A84ED1F1AB4F86D0040BA00EE41
:100C6000100AB8EE400A84ED200AB4F86F0040BACA
:100C7000A4F874002178092901D00A290BD1FFF7C3
:100C800038FC9FED091B53EC112BFFF740FBFFF7DE
:100C90005CFCA4F87400204600F0A4FF002084F857
:100CA000720010BD0000C8422DB29DEFA7C6E73FFD
:100CB0002DE9FE4F00273C4602A96846029700F046
:100CC0002DF9834A0299DFF80CB2914261D19DF867
:100CD0000100FF2811D0F02859D19DF800007E4D69
:100CE0007E4C0F284FD2DFE800F04E0B11174E4E0E
:100CF0004E1D23292F353B3E46000D20784945E007
:100D0000684601F05BFC85ED000A3CE0684601F0B6
:100D100055FC85ED010A36E0684601F04FFC85ED93
:100D2000020A30E0684601F049FC84ED030A2AE03B
:100D3000684601F043FC84ED020A24E0684601F0B5
:100D40003DFC84ED040A1EE0684601F037FC84EDAA
:100D5000010A18E0684601F031FC84ED000A12E057
:100D600001F0BCFF0FE0684601F028FCBDEEC00AB0
:100D70008BED000A07E0684601F020FCBDEEC00ADA
:100D8000584880ED000A9DF8000057490870BDE8FA
:100D9000FE8F564A9142FAD10DEB0008544E18F8D6
:100DA000011CDFF85091544D6A46CB0906D02F70D4
:100DB00089F8007001F01F030224337096F800C018
:100DC00001F01F034D4E634526D1C1F3401C99F835
:100DD00000108C4520D139B1002189F80010484B12
:100DE0009246A0F1010C15E00121F6E729785A6836
:100DF000914200DD59600C2905D908F8017C2F705B
:100E000089F8007008E01AF804207254491C641C28
:100E10002970E4B26445E9DB18F8011C4906B6D52F
:100E20000828B4D128780C284DD101F0A1F9DBF8BD
:100E300000000028B08800D0404201B2314890F84C
:100E4000A80010B92F4801F025FC264800680028AA
:100E5000F08800D0404201B22B4890F8A80010B9A9
:100E6000294801F017FC70884FF4FA6801B201F5C7
:100E70007A7040450DD8254C94F8A80048B9204612
:100E800001F008FC94F98910B4F9040001F08EF81F
:100E9000E083308801B201F57A7040450DD81C4CD2
:100EA00094F8A80048B9204601F0F4FB94F98910A1
:100EB000B4F9040001F07AF8E0831649308908801B
:100EC0001549708908802F7089F800705FE700006D
:100ED0000A574E01280000208803002094030020B8
:100EE000020000202C000020010000200A554E01C5
:100EF000860000208500002084000020C003002020
:100F00008800002018020020D0020020A800002045
:100F100060010020040000200600002070B50F4E84
:100F20000D46044686B00021304600F074F90028D2
:100F300012D06A460021304600F0D5F901982860A9
:100F40000021684603E04218D27A6254491C9DF899
:100F50000A208A42F7D8D0B206B070BD00640040C3
:100F6000F0B585B00023CDE9003104218DF80810DB
:100F70008DF809308DF80A20694604E0C45CCD186C
:100F80005B1CEC729BB29342F8D30C4F384600F0D6
:100F9000F1F90646002440F6FF7501E0641CA4B296
:100FA0003146384600F038FA08B9AC42F6D3AC42C4
:100FB00002D3012005B0F0BD0020FBE70064004033
:100FC00038B50F4D09240B234FF400622946012048
:100FD000009400F083F80C23AA1429460120009401
:100FE00000F07CF801220621142000F06EF901B017
:100FF0002802BDE83040034B034A044900F016B90B
:10100000000002400A574E010A554E01006400409C
:10101000F0B5827A2F4D012191402A6842F00102F9
:101020002A602C4E1C3632688A433260294A047B7F
:10103000294B0C32A4B914688C4314604488C788C7
:1010400044EA0744877A03EBC707C7F84046048899
:10105000878844EA0744877A03EBC707C7F8444602
:10106000047B012C12D114680C431460847A02684A
:1010700003EBC4044FEA3242C4F84026847A426843
:1010800003EBC4034FEA3242C3F84426114AC37A41
:10109000121D002B136806D00B4313600D4A038901
:1010A000143213B104E08B43F7E713688B431360EA
:1010B0000389012B02D113680B431360407B012885
:1010C00002D1306808433060286820F001002860B1
:1010D000F0BD000000660040006000402DE9FC41CA
:1010E0000D461F4614460121089E01F0EBF93246D9
:1010F0003946284600F041FF02218DF804100021F6
:101100008DF8061003208DF8050001208DF80700EA
:1011100000946946284600F0F4FEBDE8FC81002AF0
:10112000426901D00A4300E08A434261704710B52A
:101130000368002223F002030360036843F0010305
:1011400003604FF6FF7300E0521C4468E40701D1CE
:101150009A42F9D14268D2073ED08A79012A0268C0
:101160003CD022F080020260CA79012A026838D09D
:1011700022F0400202600A7A012A026834D022F08A
:10118000200202604A7A012A026830D022F010025E
:1011900002608A7A012A02682CD022F008020260DA
:1011A000CA7A012A026828D022F0040202608A78F2
:1011B000CC78920742EA04620C7942EA04424C7904
:1011C000098842EA0452491E0A43C261016821F0BB
:1011D00001010160002114E0002010BD42F08002F6
:1011E000C1E742F04002C5E742F02002C9E742F001
:1011F0001002CDE742F00802D1E742F00402D5E741
:10120000491C4268D20701D09942F9D14068C00711
:10121000E2D1012010BD0246002029B1012902D1EE
:10122000106900F003007047D068FAE72DE9F0413B
:10123000884688B01E461746012101F04FF9002468
:101240008DF806408DF8074007208DF80400042033
:101250008DF8084001258DF802408DF805008DF8C5
:1012600009508DF8034006208DF80A40ADF80000C3
:101270008DF80B4069464046FFF759FF780BADF8F3
:101280000C004FF6FF7000EAC701091DADF80E1003
:10129000710B00EAC6008DF81640ADF81010001D65
:1012A0008DF817508DF81850ADF81200ADF81440B5
:1012B0008DF8195003A8FFF7ABFE0122022140462A
:1012C000FFF72DFF08B0BDE8F08108B58DF80000EC
:1012D0008DF801108DF8022001208DF8030068467A
:1012E00001F0AAF808BD10B500EB0113D3F8B04126
:1012F00014F004041472D3F8B04133D0E4085460FD
:10130000D3F8B04104F002045472D3F8B44104F0AD
:101310000F049472D3F8B441240AD474D3F8B841BA
:10132000D472D3F8B841240A1473D3F8B841240C0A
:101330005473D3F8B841240E9473D3F8BC41D473DA
:10134000D3F8BC41240A1474D3F8BC41240C54745F
:10135000D3F8BC311B0E937439B1016941F02001FF
:10136000016110BD640D1460CAE7C16841F020013D
:10137000C16010BD30B50246002093685B0108D4FF
:101380009068000101D5012003E09068C00037D5C6
:10139000022002EB0012D2F8803103F00103C2F800
:1013A00080310B7A73B3D2F880414D681C434B7A7D
:1013B00043EAC5031C43C2F880418B7A03F00F0354
:1013C0008B72D2F8843123F00F03C2F88431D2F843
:1013D00084318C7A2343C2F88431CB7ACC6843EAD7
:1013E0000423C2F88831CB7B096943EA0121C2F8A2
:1013F0008C11D2F8801141F00101C2F8801130BD8A
:10140000042030BDD2F880314C7A23430C8843EA63
:101410004453C2F88031D0E7002221B1012905D020
:10142000022906D112E08268114801E08268114861
:1014300002401149501A8A4214D00ADCA2B16FF05E
:10144000806010180FD002280CD10FE082680B4882
:10145000EEE7B0F5007F09D00949401803D0B0F598
:10146000003F03D0002070470220704701207047E2
:10147000030000040003000800010008000003103E
:101480000001FFF770B5094D094C2946204600F0D0
:1014900007FA002809D02946204600F02BF92046FB
:1014A000BDE87040002100F03BB970BD2080001005
:1014B0001060024070B5094D094C2946204600F0E5
:1014C000EFF9002809D02946204600F013F92046FC
:1014D000BDE87040002100F023B970BD0080001805
:1014E0005860024070B5094D094C2946204600F06D
:1014F000D7F9002809D02946204600F0FBF82046FD
:10150000BDE87040002100F00BB970BD00880020DC
:10151000886002402DE9F05F624D634C29462DED55
:10152000028B204600F0BCF900287CD029462046DA
:1015300000F0E0F8204600F0ABF95C49002873D0D9
:101540005B485D4BDFF874A102880A8042884A80BC
:1015500082888A80C288CA8002890A81554A408965
:1015600048815088401C80B250804D88D3F890400C
:10157000B0F5C87F04EB050CC3F890C0CE88DAF84C
:1015800090504F4C2E44CAF8906054F8905F0F88EA
:101590003D444C4F2560B1F8048057F8904F4444C7
:1015A000A1463C60484C0F89D4F80080474427602E
:1015B000464C4989D4F800804144884621606AD36A
:1015C00000EE10CA42490120B8EE400A087000241B
:1015D00054809B469FED3F8A20EE080A10EE100AC9
:1015E000FEF7CCFF00EE106ACBE92601B8EE400A08
:1015F00020EE080A10EE100AFEF7C0FF00EE105AA7
:10160000CAE926012E4EB8EE400A20EE080A10EE76
:10161000100AFEF7B3FF00EE109A2A4DB8EE400A0A
:1016200020EE080A01E036E039E0C6E9260110EEB6
:10163000100A9036FEF7A2FFC5E9260100EE107AE7
:10164000CBF89040CAF89040B8EE400A3460C5F834
:1016500090401D4D10EE100AFEF790FF9FED1E1BEF
:1016600053EC112BFEF753FE9FED1D1B53EC112B7A
:10167000FEF7BFFEFEF7C6FF1B4908604FF4C871B6
:10168000B8FBF1F02C60114D80B200F0DDFC174882
:1016900080ED000A2C60BDEC028BBDE8F09F144881
:1016A0004FE700002080001010640240CC030020AF
:1016B000B403002088000020A80000206001002062
:1016C00018020020D00200203800002090000020E6
:1016D00003000020ACC5273843CA4FAA7D3A0A4010
:1016E000000000000000F94034000020300000201D
:1016F000A8030020074A904201D2074801E00548AC
:101700001038064A8B0001EA020101D5C16070471A
:101710008160704710640240006002407D0F7D0FC1
:101720000029016802D041F0010101E021F001012E
:10173000016070472DE9F043016821F0010101606B
:101740000021016041608160C1600161212141612E
:101750003C493C4A3D251039904202D18D60BDE89C
:10176000F083384A4FF474661832904201D18E608B
:10177000F5E7344A4FF474173032904201D18F604C
:10178000EDE7304A4FF0746C4832904202D1C1F814
:1017900008C0E4E72B4B2C4A6033984201D1CA6061
:1017A000DDE7284C294B7834A04201D1CB60D6E745
:1017B000DFF89080264C08F19008404501D1CC60BC
:1017C000CDE7DFF880804FF03D5908F1A80840458B
:1017D00002D1C1F80C90C2E71E49DFF878800839C1
:1017E000404501D10D60BAE71A4D1835A84201D124
:1017F0000E60B4E7174D3035A84201D10F60AEE757
:10180000144D4835A84202D1C1F800C0A7E7114DD8
:1018100010496035091FA84201D10A609FE70D4AAF
:101820007832904201D10B6099E70A4A9032904297
:1018300001D10C6093E7074AA83290428FD1C1F8DA
:1018400000908CE7106002403D000020400F002017
:1018500000003D20106402400029016802D041F4DC
:10186000802101E021F4802101607047002A026894
:1018700002D042F4002201E022F400220260016161
:101880007047014600200968C90700D00120704751
:10189000014600200968090300D5012070470000B7
:1018A00030B5104A0024904201D20F4A01E00D4A9F
:1018B000103A0E4B194205D01E2303EAD1250368C6
:1018C0002B4002E0406900F08003880001D5506899
:1018D00000E01068064A1040084201D003B101241C
:1018E000204630BD10640240006002403C0F3C0FB7
:1018F0007D0F7D0F0B0607D5436912B143F08003BE
:1019000001E023F080034361802908D0002A0268A7
:1019100001F01E0101D00A4300E08A4302607047D3
:1019200030B50368124ACC6813400A682243D1E9F3
:1019300005452C432243CC6922430C6A22434C6A5E
:1019400022438C6A22434C6B22438C6B22431A4302
:101950000260426922F00703D1E90B2422431A43B3
:1019600042610A6942604A6882608968C16030BD2C
:101970003F801CF02DE9F0438FB08846DDE9166505
:10198000814601211C461746480500F09BFD38465C
:10199000FFF7D0FE3846FFF774FF0028FAD1402049
:1019A000CDE902501220049000204FF48061CDE96F
:1019B0000501890007918900CDE908108900CDE96A
:1019C0000A100321CDE90C10CDE900460E906946BE
:1019D0003846FFF7A5FF01224146484601F0CEFBFD
:1019E00010213846FFF786FE012210213846FFF706
:1019F00081FF00213846FFF793FE0FB0BDE8F0836A
:101A00002DE9FE4F01263A4F052320223946304664
:101A1000009600F083F8DFF8E0A04524CDE9004A05
:101A2000DFF8D0800323A20701213448CDF80880D5
:101A300000F0A3F800221146102000F090F80225D3
:101A40000723802239460120009500F067F8DFF86F
:101A5000B0902C4F8DE8900203232B4A0221274897
:101A600000F08BF800221146102000F078F8DFF823
:101A70009CB00723802259460220009500F04EF8C2
:101A80008DE89002224F03233A4604211B4800F0C0
:101A900074F8002211460E2000F061F8062340225F
:101AA00059460220009500F039F8CDE9004A032399
:101AB0003A4604211148CDF8088000F05EF8002273
:101AC00011460B2000F04BF840F28F11CDE90016C3
:101AD0000020029053230F4A01210F4801F06AFBB6
:101AE00003B00022BDE8F04F0121192001F089BBAD
:101AF000000002408132000821320008DD24000885
:101B00000D3300088D32000800040040000402403C
:101B10000008004000000140F52400082DE9FC41C8
:101B20000D461F4614460121089E00F0CBFC3246AC
:101B30003946284600F021FA02218DF804100321CD
:101B40008DF8051000208DF8060001208DF80700A3
:101B500000946946284600F0D4F9BDE8FC8108B538
:101B60008DF800008DF801108DF8022001208DF80D
:101B70000300684600F060FC08BD2DE9F041904686
:101B800088B002460EA81C4690E8E0000B460121F2
:101B900018469047ADF800400024ADF80840ADF875
:101BA000024001958DF80A406946404601F0C0FBAD
:101BB0006020ADF80C000120ADF80E000594ADF8E2
:101BC000184003A94046B04708214046B8470121C4
:101BD000404601F0B1FA0121404601F0BAFA08B0DE
:101BE000BDE8F081B0F874100D4A00EE101AD2ED85
:101BF000030AB8EE400A92ED041A41EE000A00EE24
:101C0000101A92ED051AB8EE400A20EE011A00EE05
:101C1000101AB8EE400A41EE000AC0ED250A7047DE
:101C20000000002005490028086802D040F48060C8
:101C300001E020F48060086070470000003C024032
:101C400070B50646002529B1012927D0022928D0E0
:101C50004FF4407500F080F809281ED1124C20681E
:101C600020F440702060206828432060206820F025
:101C7000F8002060206846F00201084320602068D8
:101C800040F48030206000F067F8216821F0020104
:101C90002160216821F0F801216070BD4FF480754A
:101CA000D8E74FF40075D5E7103C02400D490920F4
:101CB0000A68D20301D5012070470A68D20601D50F
:101CC000062070470A68D20501D5022070470A68CD
:101CD00012F0E00F01D00720704709688907FBD593
:101CE000082070470C3C02400248016841F0004166
:101CF00001607047103C024070B50D46064600F08A
:101D00002BF8092813D10A4C206820F44070206079
:101D1000206840F400702060206840F001002060DE
:101D2000356000F019F8216821F00101216070BDD3
:101D3000103C024005480068002805DA03480449C1
:101D40000C3801600349016070470000103C0240FC
:101D500023016745AB89EFCD08B509208DF8000058
:101D6000FFF7A4FF8DF800009DF800000128F7D0D0
:101D70009DF8000008BD000010B5234800F0E6FC07
:101D80002249884201D000F047F81F48001D00F0AA
:101D900011FC1F4C1C4884ED000A083000F00AFCBE
:101DA000194884ED010A0C3000F004FC164884ED5B
:101DB000020A203000F0FEFB0C34134884ED030AC5
:101DC0001C3000F0F7FB104884ED020A243000F0CC
:101DD000F1FB0D4884ED040A283000F0EBFB0A48C3
:101DE00084ED010A2C3000F0E5FB074884ED000A81
:101DF000303000F0ABFC074CA0620348343000F0F8
:101E0000A5FCE06210BD0000000006087856341200
:101E1000880300200000002010B572B60122294975
:101E2000294800F095FC00F0A3F927480122274932
:101E3000001D00F08DFC254923480122091D0830B2
:101E400000F086FC21492048012208310C3000F0C6
:101E50007FFC00F08DF91D491B480122183120300C
:101E600000F076FC19491848012214311C3000F0AA
:101E70006FFC1649144801221C31243000F068FC24
:101E800000F076F91149104801221031283000F095
:101E90005FFC0E490C4801220C312C3000F058FC3C
:101EA00000F066F9084801220949303000F050FC82
:101EB000074905480122091D343000F049FC62B68B
:101EC00010BD000044000020000006088803002028
:101ED000280000207CB50D461446012100F0F2FADE
:101EE00001228DF8042000208DF8060003208DF8D3
:101EF000050000948DF807206946284600F001F897
:101F00007CBDF0B5002201274FF0030C0B6807FAE7
:101F100002F52B40AB422CD1066853000CFA03F4B7
:101F2000A64306600E79D0F800E09E4046EA0E0611
:101F300006600E79012E01D0022E12D18668A643CA
:101F400086604E79D0F808E09E4046EA0E0686602C
:101F50004668AE43466045688E799640B6B23543D2
:101F60004560C568A543C560CC799C40C3681C43E7
:101F7000C460521C102AC9D3F0BD4B07DB0E9A4037
:101F8000C90810B500EB8100016A0F249C40A143F1
:101F90000162016A1143016210BD418370470183F0
:101FA000704742694A4042617047000070B50C4674
:101FB000054610FB04F0FEF78BFA41EC100B002DE8
:101FC0000DDB51EC100B9FED121B53EC112BFEF7A8
:101FD0009EF9FEF79BFA80B240F2AE3110E09FED21
:101FE0000E1B51EC100B53EC112BFEF790F9FEF782
:101FF0008DFA0B4901FA80F0404280B240F26C71D8
:10200000884200D90846002C00D1002070BD000095
:10201000AF25E4839ECDBA3F9A9999999999B93F92
:10202000E9FBFFFF10B50C4601F0C0FBC1B294F80C
:1020300072000A2802D204F16802815414F8720F67
:10204000401C207010BD000010B52DED068B9FEDDB
:102050002D9AFEF74EFA9FED2C8B53EC182BFEF7C2
:1020600056F99FED2B1B53EC112BFEF7C2F9FEF72F
:10207000C9FA09EE900A19EE900AFEF77FFA53ECBE
:10208000182BFEF741F929EE290A41EC180B10EE46
:10209000100AFEF773FA53EC182BFEF7AAF9FEF7B5
:1020A000B1FA00EE100A9FED1C8B9FED1DABC0EE48
:1020B000090A10EE900AFEF761FA41EC100B01F0EC
:1020C00083FB53EC1A2B51EC100BFEF792F953ECF7
:1020D000182BFEF775F841EC100B53EC102B9FED0D
:1020E000120B51EC100BFEF784F99FED111B53EC12
:1020F000112BFEF706F9FEF785FABDEC068B00EE14
:10210000100A10BD0050C3476666666666660A40E0
:102110000000000000FEAF40000000E0E1796B3FEE
:102120000000000000DCAE40000000000000F03FB6
:1021300066666666660A7140FEE770B504460D463F
:1021400045F2555000F02AF8204600F01BF82846CA
:1021500000F01EF800F00EF8BDE87040AFF300800C
:1021600002494CF6CC400860704700000030004047
:10217000AFF3008002494AF6AA20086070470000C9
:1021800000300040014948607047000000300040C6
:102190000149886070470000003000400149086034
:1021A0007047000000300040012202492020FFF764
:1021B00091BE0000001402404FF40042014920206B
:1021C000FFF788BE0014024010B50C494FF0E02321
:1021D00048689A694C68A042FAD1096801EB41034A
:1021E000C3EBC113C2EBC302B2FBF1F100EB40023F
:1021F000C2EBC01001EBC00010BD00003C0000208D
:1022000070B52D4E00242DED028BF07801284DD1B4
:102210002A4D0020F07095ED260B9FED298B641C54
:10222000E4B253EC182B51EC100B9835FEF76FF815
:1022300095ED021B53EC112BFDF7C2FFC5E902011E
:10224000203553EC182B95ED260B983551EC100BDF
:10225000FEF75DF895ED021B53EC112BFDF7B0FF77
:10226000C5E90201203553EC182B95ED260B983566
:1022700051EC100BFEF74BF895ED021B53EC112BB4
:10228000FDF79EFFC5E90201203553EC182B95EDB3
:10229000260B983551EC100BFEF739F895ED021B23
:1022A00053EC112BFDF78CFFC5E90201642CACD374
:1022B000BDEC028B70BD000000000020A8000020D3
:1022C0007B14AE47E17A843F70B5B0F9043040F238
:1022D0001744002A75D0B0F97420C280058913FB19
:1022E00005F600259FED431A002E08DA002A06DDC8
:1022F000858080ED031A80ED041A058104E00381D6
:10230000002B01DD9A1A02E0B0F904301A4400EE05
:10231000102AB8EEC00A80ED030AD0ED040A91ED50
:10232000002A828B70EE601A61EE821A91ED012A0A
:1023300042EE001AB0EE002A00EEC20AD0ED050A05
:1023400030EE200AD1ED020A40EE801ABDEEE10A1D
:1023500010EE101A114409B28183B0F90420002A4A
:1023600003DB002903DC002101E00029FBDA133242
:102370008183272A07D2858380ED031A80ED041A12
:1023800080ED051A03E0B0F91C10A14201DAB0F9A2
:102390001C40194984838C4200DC0C468483002C49
:1023A00004DAA4F217446142C18300E0C48390EDD3
:1023B000040A80ED050A90ED030A80ED040A70BD61
:1023C000FFE7002B08DB03EB4301890009B2C1835F
:1023D000A142F4DBC483F2E7A3EB83014FF48362F1
:1023E00002EB810109B240F2FF72C1839142E6DB48
:1023F000C283E4E70000000018FCFFFF0B4810B5A3
:10240000C178012911D10021C170094800F07AFC7E
:102410000748B83000F076FC064800F073FC054829
:10242000BDE81040B83000F06DBC10BD00000020C9
:10243000A80000201802002030B50F23C2780178D0
:102440000125FAB1144A126801F1E02102F4E062B8
:10245000C2F5E062C2F30722C2F10404D34042781D
:10246000A24084781C401443220181F800240078A3
:1024700000F01F018D404009800000F1E020C0F80D
:10248000005130BD01F01F0085404809800000F177
:10249000E020C0F8805130BD0CED00E00249084357
:1024A00002490860704700000000FA050CED00E0EA
:1024B00003484078002801D000F048BB7047000076
:1024C00000000020044A0029116801D0014300E007
:1024D000814311607047000030380240044A0029EF
:1024E000116801D0014300E0814311607047000092
:1024F00040380240044A0029116801D0014300E03D
:10250000814311607047000044380240044A0029AA
:10251000116801D0014300E0814311607047000061
:102520002438024070B5204B1968204C11F00C0182
:1025300004D06610042903D0082903D004601BE0EE
:10254000066019E0184A121F1168C1F3805511681E
:1025500001F03F0115B1B6FBF1F101E0B4FBF1F17F
:1025600014681268C4F388146143C2F30142521C18
:102570005200B1FBF2F1016019680F2202EA111159
:102580000B4A545C0168E14041601C68072505EA7C
:102590009424145D21FA04F484601B6805EA533323
:1025A000D25CD140C16070BD083802400024F40004
:1025B0009400002090ED000A7047000070B50446BA
:1025C0002DED048B857905F00F00FDF792FF9FED4F
:1025D0002C1B53EC112BFDF79AFE41EC180B28092C
:1025E000FDF787FF9FED281B53EC112BFDF78FFEA6
:1025F00041EC190BA078264A0109514300F00F0065
:1026000043F6095210FB02F001EB8011E07840F62E
:102610003543020912FB03F201EB421100F00F00F7
:1026200040F2712210FB02F001EB0012217908093F
:1026300000EB4003C3EBC01002EBC00201F00F003F
:1026400000EBC00101EB001002EB80026079010990
:1026500001EB810102EB410100F00F000844FDF79E
:1026600037FF53EC192BFDF7ABFD53EC182BFDF79F
:10267000A7FDFDF7C7FFBDEC048B00EE100A70BD8F
:102680007B14AE47E17A843F9A9999999999B93F19
:1026900080969800B0F90820002A03DA002901DBAF
:1026A0008188891C81800181704700001C49884213
:1026B00001D2002070471B49884201D20820704790
:1026C0001949884201D2102070471849884201D226
:1026D000182070471649884201D2202070471549BA
:1026E000884201D2282070471349884201D2302005
:1026F00070471249884201D23820704710498842F9
:1027000001D2402070470F49884201D248207047CB
:102710000D49884201D25020704758207047000070
:10272000004000080080000800C000080000010808
:102730000000020800000408000006080000080865
:1027400000000A0800000C0800000E08006870472E
:102750002DE9F04104461D48092690460F46844263
:1027600031D3A0072FD1FFF7E5FA0020FFF75AFA7F
:102770001748254604EB880884420ED31AE02868DF
:10278000401C09D02846FFF791FF0221FFF758FAB5
:102790000646092801D00FE02D1D4545EFD3092E2F
:1027A00008D009E020463968FFF7A6FA092803D1C6
:1027B000241D3F1D4445F5D30120FFF733FABDE842
:1027C000F041FFF791BABDE8F08100000000060873
:1027D0000000FF1F174A30B4174832F8741FA0F1E9
:1027E0000C03017092F91520090AC2F10A0241EAAC
:1027F0000211124A417032F8741F817092F915204B
:10280000090AC2F10A0241EA0211C17000220271F2
:1028100042718271D97801F1C004C471491CC8B2F7
:10282000D870202800D3DA7030BC0822044902484E
:10283000FEF796BB6001002054000020A800002095
:1028400001534E1F30B40E48002103220170417025
:102850008170C17001714171A0F114048271E2783C
:1028600002F1C003C371521CD0B2E070202800D323
:10287000E17030BC082203490148FEF771BB00003B
:102880005C00002001534E1F30B413480022134B4C
:10289000027042708270C27033F8741F017193F934
:1028A0001530090AC3F10A0341EA031141710621F7
:1028B000A0F11C048171E17801F1C003C371491CCE
:1028C000C8B2E070202800D3E27030BC082204496E
:1028D0000148FEF745BB00006400002018020020FC
:1028E00001534E1F134A30B4134832F8741FA0F13D
:1028F0002403017092F91520090AC2F10A0241EA83
:102900000211417000228270C2700271427109216D
:102910008171D97801F1C004C471491CC8B2D87062
:10292000202800D3DA7030BC082204490248FEF7A0
:1029300017BB0000D00200206C00002001534E1F86
:102940001B48F2EE040A90ED000A1A4820EE200A15
:10295000A0F12C02BCEEC00A10EE101A017010EEAD
:10296000101A090A4170144991ED000A20EE200A5C
:10297000BCEEC00A10EE101A817010EE101A090A8F
:10298000C1700E4909880171090A41710C218171D8
:10299000D17801F1C003C371491CC8B2D07020289E
:1029A00001D30020D070082205490248FEF7D8BAAA
:1029B00034000020740000203000002008000020B7
:1029C00001534E1F104830B4018810480022A0F176
:1029D00034040170090A41700D4909788170C27090
:1029E000027142710F218171E17801F1C003C3715D
:1029F000491CC8B2E070202800D3E27030BC082225
:102A000004490248FEF7ACBA040000207C00002014
:102A10000600002001534E1F1F4AFDEEC00A107031
:102A200010EE900A51701D49F8EEE00A90FBF1F3A8
:102A3000937090FBF1F301FB130042F2107190FBD5
:102A4000F1F3D37090FBF1F301FB1300642190FBD1
:102A5000F1F330EE600A1371DFED110A90FBF1F330
:102A600020EE200A01FB13005071BDEEC00A111FB9
:102A700010EE100A9071C87800F1C003401CC0B27B
:102A8000D371C870202801D30020C87008220549DE
:102A90000148FEF765BA00004C00002040420F00DC
:102AA0000000C84201524E1F10B5264C2649A2789C
:102AB00001F10C00121F0A2A11D2DFE802F0050A08
:102AC000161B20252A2F343B91ED000AF12101200D
:102AD00003E091ED010AF1210220FFF79DFFA078AC
:102AE000002801D0401EA07010BD91ED020AF12116
:102AF0000320F2E790ED030AF1210720EDE790EDC6
:102B0000020AF1210820E8E790ED040AF1210920EA
:102B1000E3E790ED010AF1210A20DEE790ED000ADB
:102B2000F1210B20D9E794ED0A0AF1210D20B8EE2E
:102B3000C00AD2E794ED0B0AF1210E20B8EEC00ACC
:102B4000CBE70000000000208803002010B5FFF74D
:102B500063F9254C2549627801F10C000F2A14D243
:102B6000DFE802F013080D161313131B20252A2F7C
:102B700013343B0091ED000AF121012003E091EDB7
:102B8000010AF1210220FFF747FF0020607010BD0D
:102B900091ED020AF1210320F5E790ED030AF121FE
:102BA0000720F0E790ED020AF1210820EBE790ED15
:102BB000040AF1210920E6E790ED010AF1210A203B
:102BC000E1E790ED000AF1210B20DCE794ED0A0A21
:102BD000F1210D20B8EEC00AD5E794ED0B0AF121E2
:102BE0000E20B8EEC00ACEE70000002088030020C7
:102BF0000CB50022274900920192086840F4803009
:102C000008604FF4A043086800F400300190009879
:102C1000401C0090019810B900989842F3D10868C0
:102C2000800334D5012001901A484030026842F0F8
:102C3000805202601848026842F44042026015481F
:102C4000083002680260026842F4004202600268D2
:102C500042F4A0520260031F104A1A600A6842F050
:102C600080720A600A689201FCD50D4940F2057233
:102C70000A60016821F003010160016841F002016E
:102C800001600168C1F381010229FAD10CBD0192F2
:102C90000CBD00000038024000700040085440079E
:102CA000003C024000F8041B002120F8851B0A228A
:102CB00000F819299FED070B01764183818380ED90
:102CC0000C0B022280F83A20818780F8381080F8B7
:102CD000421070470000000000000000012080F357
:102CE0001388BFF34F8F05480168054A01F4E0617E
:102CF00011430160BFF34F8F00BFFDE70CED00E013
:102D00000400FA052DE9F04704462DED028BB0F8DA
:102D10007400634D00EE100AD5ED040AB8EE400AC7
:102D2000B4EEE00AF1EE10FA02DB95ED020A01E0E2
:102D300095ED030A2178DFF86C91012794F9A8003A
:102D400000264FF0FF3809293ED200287AD194EDB1
:102D5000251AF6EE000A41EE000A10EE900AFDF781
:102D60000DFC94ED281B94ED260B41EC180B53EC55
:102D7000112B51EC100BFDF7C4FA53EC182BFDF797
:102D800029FC1BD2B4F88C00401C80B2A4F88C0043
:102D9000502811D39FED440B84ED260BA4F88C60D2
:102DA00094F98900002805DD401E40B284F88900AE
:102DB000012801DA84F88960686836E0A4F88C603C
:102DC000FAE784F8A88056E0E0BBE06FFDF7D6FB99
:102DD00094ED261B53EC112BFDF799FA9FED341B54
:102DE00053EC112BFDF7F6FB17D2B4F8AC004FF6FD
:102DF000FF71401C80B2A4F8AC0088420DD395ED61
:102E0000000AF3EE090A80EE201ABDEEC10A10EEA8
:102E1000100A07FA80F0A4F8AC0095ED010AF1EE73
:102E2000040A30EE600A10EE100AFDF7A7FB94EDDD
:102E3000261B53EC112BFDF7B5FBC2D994F8A80063
:102E4000002828D094F9A800002813DDA0F1010083
:102E500040B284F8A800D8B92078A0F1010007FAA0
:102E600000F7B9F8080020EA0700A9F8080084F87C
:102E7000B2600DE00CDA84F8B2702078B9F808106E
:102E8000A0F1010007FA00F747EA0107A9F8087066
:102E9000A680E683A683BDEC028BBDE8F087000028
:102EA000940300200000002000000000000000004B
:102EB0000000000000E08540144810B50268144985
:102EC0000B6AD21A142A20D3006808620878421CC0
:102ED0000A70032801D300200870087848B101283F
:102EE0000DD0022811D1FFF72BFDBDE81040FFF7F0
:102EF00069BDFFF76FFCBDE81040FFF7A3BCFFF70B
:102F0000C3FCBDE81040FFF7EDBC10BD4000002041
:102F10000000002005490A6805488369D21A0A2A78
:102F200003D309688161FFF7BFBD704740000020EF
:102F3000000000200C4900B50A680C48C369D21A89
:102F4000142A0FD30968C16109490022A1F5B8709C
:102F5000FFF7BAF906490022A1F1B8005DF804EBC9
:102F6000FFF7B2B900BD00004000002000000020C3
:102F70008803002070B514480168144C626A891AED
:102F8000B1F5FA7F1FD30068114D60620121284618
:102F9000FFF707F8A0884FF400460028314628467E
:102FA00002D0FEF7FAFF01E0FEF7F9FFE1880948D9
:102FB0000029314603D0BDE87040FEF7F0BFBDE800
:102FC0007040FEF7EABF70BD400000200000002006
:102FD000001402400000024002480168491C0160E0
:102FE0007047000040000020124810B5016841F40D
:102FF000700101601048016841F0010101600E4A52
:1030000000210832116002680C4B1A400260031D57
:103010000B4A1A60026822F48022026006480C30D3
:103020000160FFF7E5FD03494FF00060803908605B
:1030300010BD000088ED00E000380240FFFFF6FE02
:10304000103000242DE9FC41314C0121204600F0D4
:103050009DF8002859D00121204600F077F82D492D
:103060000878421C0A70042801D3002008700878F0
:103070004FF08063284E5914D8B1284D4F000128D5
:1030800025D0022832D003283FD1254C2548CDE950
:1030900000044FF0C0632A460007FEF76BFCA4F162
:1030A00020002A46C18B02B02046BDE8F04100F066
:1030B000BFBE19481C4C3430184DCDE90004783D92
:1030C0002A463046FEF756FCA4F12000E9E7174CEB
:1030D0001748CDE9000416484FF020632A463946C8
:1030E0003838FEF747FCA4F12000DAE70A48114C13
:1030F00038300A4DCDE90004303D2A463946304685
:10310000FEF738FCA4F12000CBE7BDE8FC8100000D
:103110000000014088000020000800408860024054
:10312000380200203400004080010020C800002048
:1031300038040040F00200200029018802D041F04C
:10314000800101E021F0800101807047C9430182C4
:1031500070470029018802D041F0010101E021F00F
:10316000010101807047002930F8441F02D041F46A
:10317000004101E0C1F30E0101807047002A8289FD
:1031800001D00A4300E08A43828170470246002052
:10319000138A92890B4202EA010202D0002A00D06F
:1031A00001207047002A828901D00A4300E08A4347
:1031B00082817047FEB517460A4605461C46012126
:1031C0001046089EA8470020ADF80040ADF8020068
:1031D000ADF8080001966946384600F0A9F80121CB
:1031E0003846FFF7A9FF2021384600F099F8012260
:1031F00011463846FFF7D6FF01213846FFF7A9FFF1
:10320000FEBD08B58DF800008DF801108DF8022084
:1032100001208DF803006846FFF70EF908BD000095
:1032200030B5028C22F001020284028C8388048B68
:1032300022F0020224F073050C882C438D8915437B
:103240004A882A430C4DA84202D00C4DA8420DD109
:1032500022F00805CA8923F440732A4322F00405AA
:103260008A882A430D8A1D434B8A2B43838004831B
:1032700089684163028430BD0000014000040140C0
:10328000028B22F008020A430283704770B5028C59
:1032900022F010020284028C8388048B0D8824F4AF
:1032A000E6464FF6FF7404EA052535438E8922F081
:1032B000200204EA061616434A8804EA0212324340
:1032C000104EB04202D0104EB04215D122F080060E
:1032D000CA8923F4406304EA0212324322F0400612
:1032E0008A8804EA021232430E8A04EA86061E43E2
:1032F0004B8A04EA830333438380058389688163AF
:10330000028470BD0000014000040140028B4FF6B2
:10331000FF7322F4006203EA012111430183704725
:10332000828822F07002828082880A4382807047FD
:1033300030B50288164C174DA0420DD0A8420BD0D4
:10334000B0F1804F08D0144B984205D0134B9842EF
:1033500002D0134B984203D122F070034A881A43DB
:10336000104B984206D0104B984203D022F4407381
:103370000A891A4302804A68C2620A880285A0420A
:1033800001D0A84201D1897A01860121818230BD14
:10339000000001400004014000040040000800401B
:1033A000000C0040001000400014004070B5104CAC
:1033B00040F225552946204600F032F948B10D4922
:1033C0002046FEF72FFE29462046BDE8704000F05B
:1033D0008BB840F22441204600F022F9002806D0A4
:1033E0002088A088BDE870400248FDF711BC70BD80
:1033F000005000406001002070B5114C40F225558E
:103400002946204600F00CF948B10E492046FEF747
:1034100009FE29462046BDE8704000F065B840F23C
:103420002441204600F0FCF8002808D020880448F9
:10343000001D0088BDE870400248FDF7E9BB70BD83
:10344000004400401802002070B5114C40F2255590
:103450002946204600F0E4F848B10E492046FEF720
:10346000E1FD29462046BDE8704000F03DB840F23D
:103470002441204600F0D4F8002808D020880448D1
:10348000001D0088BDE870400248FDF7C1BB70BD5B
:1034900000480040A800002070B5114C40F22555AE
:1034A0002946204600F0BCF848B10E492046FEF7F8
:1034B000B9FD29462046BDE8704000F015B840F23D
:1034C0002441204600F0ACF8002808D020880448A9
:1034D000001D0088BDE870400248FDF799BB70BD33
:1034E00000140140D00200200A0A01219140C94382
:1034F000018070470029818902D041F4005101E028
:1035000021F400518181704738B5032000900823D1
:10351000294A0721012000F063F800220321262018
:1035200000F036F94FF4E1342346244A4FF40031D9
:10353000234800F003F90B2000904FF40063214A68
:103540000721022000F04CF800220321272000F080
:103550001FF923461C4A4FF48021194800F0EEF869
:103560000220082100900423184A084600F038F889
:1035700000220321352000F00BF92346144A4FF4B2
:1035800080110F4800F0DAF8092000904FF4007322
:10359000104A0821402000F023F800220321472090
:1035A00000F0F6F801B02346BDE830400A4A202179
:1035B0000A4800F0C3B80000000002400044004088
:1035C000DD2400080004024000480040000C0240D6
:1035D000005000400018024000140140F52400088B
:1035E0002DE9FC410E461C4615460121089FFEF7B9
:1035F00069FF324639462846FEF7BFFC02218DF8A6
:1036000004108DF8051000208DF8060001208DF8BB
:103610000700009469462846FEF773FCBDE8FC816C
:1036200070B501F01F0501260024C1F3421306FA0C
:1036300005F2012B0FD0022B0FD0838A4FEA112104
:103640000088134206FA01F600EA060001D000B134
:103650000124204670BD8389F0E7038AEEE710B5A8
:10366000C1F3421301F01F040121A140012B07D037
:10367000022B07D01430002A026805D00A4304E068
:103680000C30F8E71030F6E78A43026010BD000006
:103690007FB50446008A0D46C98820F44050014396
:1036A0002182A08941F20C618843A9882A891143AB
:1036B0006A8902431143A181A08A20F44071A8893C
:1036C0000843A0826846FEF72DFF1A48844202D0C4
:1036D0001948844201D1039800E00298A1890904A5
:1036E00000EBC00101EB0010296801D5490000E0A2
:1036F0008900B0FBF1F06422B0FBF2F109010B0983
:103700006FF018056B4300EB8300A3891D044FF095
:10371000320306D503EBC000B0FBF2F000F0070067
:1037200005E003EB0010B0FBF2F000F00F000843DF
:1037300020817FBD00100140001401407FB5164676
:103740000A4605461C4601211046A8470020ADF850
:103750000800ADF804000421ADF80600ADF80A1029
:10376000ADF80C00009469463046FFF791FF012246
:1037700040F225513046FFF772FF012240F224410A
:103780003046FFF76CFF01213046FFF7B3FE7FBDE7
:1037900008B58DF800008DF801108DF80220012089
:1037A0008DF803006846FEF747FE08BD8088C0F329
:1037B000080070474FF4004201490120FEF78ABB20
:1037C000000002400000000070B5D94B00242DED30
:1037D000020B2DED108BDDE91010984205DA20F078
:1037E00000429A4201D809D141B19DED100BBDECC8
:1037F000108B02B0BDE8704000F05EBAB0F5801FDB
:1038000026DA11430BD0002813DA012000F080FAE9
:10381000BDEC108B02B0BDE8704000F059BA022038
:1038200000F076FA00F030FA51EC100B81F0004114
:103830009EE06FF035049FEDC00B53EC102B9DED17
:10384000100B51EC100BFCF762FDCDE9100108469E
:1038500004EB2051C0F31304B948A1F2FF31204416
:1038600000F4801080F07F6282F04052224301EB2E
:1038700020559FEDB50B119253EC102B9DED100BC5
:1038800051EC100BFCF73DFD41EC180BA01CC0F3F4
:1038900013009FEDAFDB9FEDB0EBB14E7E440328EC
:1038A0006CD296ED000B51EC180B53EC102BFCF77F
:1038B00079FE1DD1002D01BF96ED000BBDEC108BE4
:1038C00002B070BD2846FCF703FE41EC180B53EC28
:1038D0001D2BFCF71CFD41EC190B53EC1E2B51EC7E
:1038E000180BFCF714FD53EC192BFCF769FC3FE0B7
:1038F0009FED9D0B51EC180B53EC102BFCF707FDC3
:103900009FED9B1B53EC112BFCF7FEFC41EC190BBC
:1039100053EC182B51EC180BFCF7F9FC53EC192B5A
:10392000FCF7F5FC41EC190B002D04BF53EC192BEF
:1039300051EC180B1AD02846FCF7CAFD41EC1A0BC3
:1039400053EC1D2BFCF7E3FC53EC192BFCF7DCFCD0
:1039500053EC182BFCF7D5FC41EC180B53EC1E2B49
:1039600051EC1A0BFCF7D3FC53EC182BFCF7C9FCF9
:10397000BDEC108B02B041EC100B70BD9FED7E0BC7
:1039800051EC180B53EC102BFCF71AFC41EC100B0C
:1039900051EC180B53EC102BFCF72BFD41EC190BE1
:1039A0002846FCF795FD41EC1B0B53EC192B51EC11
:1039B000190BFCF7ACFC41EC1A0B714853EC1A2BB9
:1039C000261851EC1A0BFCF7A2FC41EC1F0B6D48BA
:1039D000C4F1510404F5D724B0EE4F0AF0EE6F0A9B
:1039E0000321784400F0D2F853EC1F2B51EC100B5C
:1039F000FCF78DFC41EC1C0B6348B0EE4F0AF0EE77
:103A00006F0A0421784400F0C1F853EC1A2B51ECF2
:103A1000100BFCF77CFC344353EC1C2BFCF7D0FB65
:103A200041EC1C0B002C4CDD9FED510B51EC180BA5
:103A300053EC102BFCF76BFC53EC182BFCF767FCDA
:103A400041EC1A0B55B353EC1D2B51EC1B0BFCF73F
:103A50005EFC41EC1D0B53EC1C2B51EC1A0BFCF7DC
:103A6000AFFB53EC192BFCF752FC53EC1D2BFCF76E
:103A7000A7FB53EC1A2BFCF747FC53EC182BFCF775
:103A800040FC41EC180B53EC1E2B51EC1B0BFCF7CC
:103A90003EFC53EC182BFCF734FC69E753EC1C2B71
:103AA00051EC1A0BFCF78CFB53EC192BFCF72FFC99
:103AB00053EC1A2BFCF728FC53EC182BFCF724FCD6
:103AC00056E735B353EC1D2B51EC1B0BFCF71FFCD9
:103AD00041EC1A0B53EC1C2B51EC180BFCF711FCAE
:103AE00053EC192BFCF713FC53EC1A2BFCF709FCD5
:103AF00053EC182BFCF705FC41EC180B53EC1E2B78
:103B000051EC1B0BFCF703FC53EC182BFCF7F9FBF7
:103B10002EE753EC1C2B51EC180BFCF7F2FB53EC8B
:103B2000192BFCF7F4FB53EC182BFCF7EDFB1FE70C
:103B30000000F07F00000000000000000000504383
:103B4000645F090000000000000000000000F03F7A
:103B5000763C7935EF39EA3D0000E0FE422EE63F43
:103B6000D006000000000000555555555555D53F6D
:103B7000000000000000E03F0000000000000040E6
:103B800086EBF9FF520500004805000070B50446B9
:103B90002DED028B4D1E00EBC500B0EE408AF0EE1D
:103BA000608A90ED000B35F0060017D053EC182B0F
:103BB00051EC100BFCF7ABFB41EC100B6D1E04EB52
:103BC000C50090ED001B51EC100B53EC112BFCF7D2
:103BD000F7FA41EC100B35F00600E7D1022D36D094
:103BE000042D1CD0062D1CBFBDEC028B70BD53EC08
:103BF000182B51EC100BFCF78AFB94ED0A1B53ECCD
:103C0000112BFCF7DDFA53EC182BFCF780FB94ED3D
:103C1000081B53EC112BFCF7D3FA41EC100B53ECBF
:103C2000182B51EC100BFCF772FB94ED061B53ECB8
:103C3000112BFCF7C5FA53EC182BFCF768FB94ED3D
:103C4000040B53EC102BFCF7BBFA41EC100B53ECBC
:103C5000182B51EC100BFCF75AFB94ED021B53ECA4
:103C6000112BFCF7ADFA53EC182BFCF750FB94ED3D
:103C7000001B53EC112BFCF7A3FABDEC028B41ECBB
:103C8000100B70BD000000009FED070B10B553EC4A
:103C9000102B9FED070B51EC100BFCF7AAFB41EC2E
:103CA000100B10BD0000000000000000000000002C
:103CB000000000000000F03F10B553EC102B51EC59
:103CC000100BFCF77DFA41EC100B10BD000000005A
:103CD0009FED050B10B553EC102B51EC100BFCF7BE
:103CE00088FB41EC100B10BD00000000000000003C
:103CF00002E008C8121F08C1002AFAD170477047B5
:103D0000002001E001C1121F002AFBD17047000012
:103D10000149086070470000A40000204FF6FF71C1
:103D200001EA40000022034611464240491C0011AE
:103D3000C9B20329F9D302F00F0040EA031080B2A0
:103D4000704700001FB56846FEF7ECFB0D49009870
:103D5000B0FBF1F00C49086001984FF47A71B0FBA8
:103D6000F1F0401EB0F1807F0AD24FF0E0214861AF
:103D7000064AF02082F8140D0020886107200861AF
:103D80001FBD000040420F003C0000200FE000E09B
:103D900030B50446FEF718FA054604EB4400C0EBC4
:103DA000C414FEF711FA401BB0EBC40FF9D330BDB9
:103DB00070B5064600200D46044606E0325D014619
:103DC000104600F0A7F8641CE4B2AC42F6D370BD14
:103DD000FCF7D2FE4FF48060FEF760FBFFF7B2FF06
:103DE000FDF7CAFFFDF70CFE40F6B830FFF7D0FF35
:103DF000FCF71CFDFEF704FAFDF7E2F8FFF784FB81
:103E0000FEF7D2F9FFF7D6FCFEF7D6F94FF47A7138
:103E10000420FEF792F9FEF7F1FAFFF77BF8FFF7BF
:103E200089F8FFF749F8FFF7A5F8FEF741FBF2E73D
:103E300070B515460446B1F5006F02D340F2FF702D
:103E400000E00846FFF76AFF010401D5342100E0D5
:103E50001A212160410401D5342100E01A2161605A
:103E6000810401D5342100E01A21A160C10401D5EB
:103E7000342100E01A21E160010501D5342100E080
:103E80001A212161410501D5342100E01A21616127
:103E9000810501D5342100E01A21A161C10501D5B8
:103EA000342100E01A21E161010601D5342100E04E
:103EB0001A212162410601D5342100E01A216162F4
:103EC000810601D5342100E01A21A162C10601D585
:103ED000342100E01A21E162010701D5342100E01C
:103EE0001A212163410701D5342100E01A216163C1
:103EF000810701D5342100E01A21A163C00701D058
:103F0000342000E01A20E0632846BDE8704001211B
:103F1000FDF706BC484000210722030602D582EACD
:103F2000400000E04000491CC9B2C0B20829F4D3E7
:103F3000704700000000000004FA97999999D93F52
:103F4000AF788E1DC571CC3F9FC678D0099AC33F0C
:103F5000935555555555E53F599322942449D23FE1
:103F6000DE03CB966446C73F44523EDF12F1C23FA8
:103F70000000000000000000983F00080000002042
:103F8000A8000000F03C000840400008A800002005
:103F900030070000003D00080000000000000000A5
:103FA00000000000EF1D953D5932C7BB0B604A3938
:103FB0000000000000000000000000000000000001
:103FC00000000000000000000000000000000000F1
:103FD00000000000000000000000000078563412CD
:103FE00000000000000000000000000000000000D1
:103FF00000000000000000000000000000000000C1
:1040000000000000000000000000000000000000B0
:1040100000000000000000000000000000000000A0
:104020000000000000000000000000000000000090
:10403000010203040102030406070809000000004E
:040000050800018965
:00000001FF
